:020000020000FC
:0200000003C338
:0200040018954D
:02000800189549
:02000C00189545
:02001000189541
:02001C00189535
:0200240018952D
:0200280087C08F
:02002C00A5C06D
:02003000189521
:02004000189511
:020044005EC09C
:02004800189509
:02004C00189505
:02005000189501
:020054001895FD
:020058001895F9
:02005C001895F5
:020060001895F1
:020064001895ED
:020068001895E9
:02006C001FC0B3
:020070001895E1
:020074001895DD
:020078001895D9
:02007C001895D5
:020080001895D1
:020084001895CD
:020088001895C9
:02008C001895C5
:020090001895C1
:020094001895BD
:020098001895B9
:02009C001895B5
:0200A0001895B1
:0200A4001895AD
:0200A8001895A9
:1000AC002FB6DF2DCE2DD63039F418607091C900E3
:1000BC007F7B7093C9001DC00E94900E7991FD2E1C
:1000CC00EC2EF09914C0D0912F01D03881F00F9202
:1000DC001F92D79F17FE02C07FEF05C0712D70389D
:1000EC0010F07FEF02C0000C771F1F900F907093E1
:1000FC00CE002FBE18952FB60260DD2009F0DA94E1
:10010C00CA9409F012C07AE0C72E0460F09B08C0B4
:10011C0000002E9B03C02E985D9802C02E9A5D9A0B
:10012C00BA9409F002C0B72E0160E3CF2FB67091DC
:10013C00E10073FF19C07091E100777E7093E100CC
:10014C0077277093E9007091EB0071607093EB006E
:10015C0070E07093EC0070E072607093ED00709141
:10016C00F00078607093F0002FBE18952FB68F9327
:10017C007091F40070FF07C070E07093E90070910B
:10018C00E80073FD0DD07091F40072FDD6D1F79B91
:10019C0004C07091F40073FD13D28F912FBE18958B
:1001AC00EF93FF937091F100709305017091F10042
:1001BC00709306017091F100709308017091F10039
:1001CC00709309017091F10070930A017091F10024
:1001DC0070930B017091F10070930C017091F10010
:1001EC0070930D017091E800777F7093E800709127
:1001FC000501F79B06C0713209F47DC0713A09F410
:10020C0070C0717619F0713009F00BC07091060155
:10021C00703041F07530A9F0763039F1793009F44D
:10022C0085C0E0C077277093F1007093F100709156
:10023C00E8007E7F7093E8007091E80072FFFCCFBD
:10024C00D6C0709108017F777093E3007091E8003D
:10025C007E7F7093E8007091E80070FFFCCF709186
:10026C00E30070687093E300C2C0709109017130B3
:10027C0029F0723069F0733021F1B4C0F79B03C0E0
:10028C00EEE2F2E202C0ECEFF2E2D491B3D0AFC0F6
:10029C00D0910C01D03049F070910D01703029F4DF
:1002AC00F79BD536F799D33420F0F79BD5E6F79921
:1002BC00D3E4F79B03C0E0E8F2E211C0EAE0F3E21A
:1002CC000EC070910801772319F4E4ECF2E206C039
:1002DC00713019F4E6EDF2E201C084C0D491F6D08D
:1002EC0086C070910601713209F07CC0E2EFF2E237
:1002FC00D7E0ECD07CC070910601703251F4709153
:10030C00E80072FFFCCF7091E8007B7F7093E800EF
:10031C0003C0723209F066C07091E8007E7F709362
:10032C00E8007091E80070FFFCCF61C0F79BC2E061
:10033C00F799C3E0C093E9007091EB007E7F709356
:10034C00EB007091ED007D7F7093ED00CA9591F7F5
:10035C0071E07093E9007091EB0071607093EB00A9
:10036C0071E87093EC0070E372607093ED00772786
:10037C007093F00072E07093E9007091EB00716083
:10038C007093EB0070E87093EC0070E37260709304
:10039C00ED007091F00074647093F000F79B14C042
:1003AC0073E07093E9007091EB0071607093EB0057
:1003BC0071EC7093EC0070E172607093ED007091D1
:1003CC00F00071607093F00077277093E9007091E2
:1003DC00E8007E7F7093E8007091E8007170E1F3A3
:1003EC00F69A05C07091EB0070627093EB00FF9170
:1003FC00EF91089570910D01772331F470910C01F8
:10040C007D1708F4D72FCC277091E80072FD94C0AB
:10041C0075917093F100DA95C395C830A9F7709176
:10042C00E8007E7F7093E8007091E8007570E1F34E
:10043C007091E80072FD80C0EF93FF938F939F93B0
:10044C005F935527F1E0E8E00E945E0B802D0E943F
:10045C005E0B902D813411F4933211F0982B41F4F2
:10046C0081E48093F10083E28093F1005FEF04C09C
:10047C008093F1000092F1000E945E0B802D0E948F
:10048C005E0B902D873321F4903011F4552321F419
:10049C000E945E0B002061F487E390E0F79B92E8EA
:1004AC000000F79B86E38093F1009093F10006C067
:1004BC00F79B01968093F1009093F1005F919F91CF
:1004CC008F91FF91EF91CCE0D45014C070910D013D
:1004DC00772329F470910C017D1708F4D72FCC27C2
:1004EC007091E80072FD28C0A89575917093F10089
:1004FC00DA95C39577E07C2349F47091E8007E7F10
:10050C007093E8007091E8007570E1F3D03041F71A
:10051C007091E800747009F00AC07091E8007E7F59
:10052C007093E800A8957091E80072FFFBCF709172
:10053C00E8007B7F7093E80008955F9372E07093FE
:10054C00E9007091E80072FF39C07091E8007B7F80
:10055C007093E80010FD32C07091F200772309F11E
:10056C00D62DC72D5091F1005993D53011F4D2E00E
:10057C00C0E06D2E7C2E6F93572D662D681430F0D5
:10058C0009F005C0791410F049F001C06D5F5919DC
:10059C006809623018F05F3B08F011606F917A9532
:1005AC0009F710FD0BC07091E8007B7F7093E80099
:1005BC0000007091E8007F777093E8005F910895D8
:1005CC005F9373E07093E9007091E80070FF14C0C2
:1005DC00707A7093E80011FF09C0C0ECD1E0709103
:1005EC000F0159915093F1007A95D9F71D7F7091B5
:1005FC00E8007F777093E8005F910895F89491E09C
:10060C009EBF9CEF9DBF88279FEF84B995B987B992
:10061C0098B98AB99BB98DB99EB980BB91BB00279B
:10062C0011272227CC24C394BC2CF1E0E0E09927BD
:10063C009193F130E8F3539A5B9A379907C0F1E044
:10064C00E8E055270E94690BED30D9F7519A59987B
:10065C000E94DD0C9927909380009CE09093810080
:10066C0092E081E7909389008093880092E09093C8
:10067C006F0090B7906890BF8EE19EE08093600011
:10068C009093600099279EBB0E94520B90931B0184
:10069C000E94950B0E94780BA895F69BFDCF0E94AB
:1006AC00800B0E94520B90931B01559A209A28980C
:1006BC00269A2E9A5D9AF1E0E4E00E945E0B00927D
:1006CC002301A895A8954427332718600E94DD0CB8
:1006DC000E94370C0E94540A0E94520EF79905C0D2
:1006EC0031D7F6F70E94940EFBCF2CD7F6F7F3D048
:1006FC00FCCF6F938F939F93982F6091110163950B
:10070C006093110197FF50C0903F29F42160217F25
:10071C0090931201DCC0973F19F56130A9F162305A
:10072C0081F097E090931001909113019093120136
:10073C00909114019093130197EF90931401207FE3
:10074C0095C096E090931001909113019093120133
:10075C0097EF90931301992790931401207F86C0F3
:10076C0090931201943FE8F0983F89F09E3F79F006
:10077C009A3F69F09B3F59F09C3F49F09F3F39F0FD
:10078C00963F29F0247F9FC097EF909312019927F1
:10079C00909313019093140195E090931001207F96
:1007AC0065C02160217F93C020FD0CC0207F9093F9
:1007BC0012019FE09093100199279093130190934D
:1007CC00140154C021FD1EC09093130199279093DE
:1007DC00140190911201913F79F0933F69F0907F51
:1007EC00903C21F0903D11F0226071C09295909355
:1007FC0010012160217F3AC092E09093100121609A
:10080C00217F34C020FF5FC022FD18C090931401DB
:10081C0023FF02C024605BC090911201923F49F00B
:10082C00903FF9F092959F70909310012160217F79
:10083C001DC093E090931001207F18C020FF43C08F
:10084C0022FF41C080911301809312018091140109
:10085C00809313019093140194E090931001297FDD
:10086C0005C094E090931001297F2860F894000053
:10087C0091E09093E900A8959091E80090FFFBCF50
:10088C009E7B9093E800909110019093F1009091D1
:10089C0012019093F100909113019093F1009091BB
:1008AC0014019093F1009091E8009E7F9093E800E2
:1008BC0000009091E8009F779093E8007894992736
:1008CC009093110104C0992790931101207F9F915F
:1008DC008F916F910895F09B05C0A8959A3509F0FA
:1008EC0008958BC0923011F0933019F40E943E069B
:1008FC00A3C09A3519F4D6D01F789EC0F0999CC02D
:10090C00963511F4F0D198C0933511F4D6D194C02A
:10091C00943508F064C0903408F026C0933219F472
:10092C000E946A0689C0943219F40E944A3F84C01E
:10093C00963219F40E94483F7FC09B3219F40E94F2
:10094C00D50B7AC09C3211F4C8D176C09D3219F403
:10095C000E94EA0B71C09D3311F4CDD16DC09F3351
:10096C0019F40E94AA0868C0903419F40E94330C40
:10097C0063C0913411F450D25FC0923411F405D29B
:10098C005BC0933419F40E94F80556C0943419F4E2
:10099C000E94AF0C51C0973419F40E9405074CC04B
:1009AC00983419F40E94B70647C09D3411F4F6D15F
:1009BC0043C09E3439F490913B01923010F00E9468
:1009CC0032073AC0903511F43DD236C0913519F446
:1009DC000E947F0731C0923511F461D22DC094353D
:1009EC0011F463D329C0973519F40E94C00624C0B2
:1009FC00983519F40E946C3F1FC0953511F4B0D096
:100A0C001BC09E3519F40E944C3F16C09F3519F43B
:100A1C000E945F3F11C09C3719F40E94C80C0CC097
:100A2C009E3719F40E94F60B07C09D3009F435C0AF
:100A3C009A3011F0903209F40895F79909C0809119
:100A4C002301806C0E947F038FE30E947F0305C00B
:100A5C008FE30E94050B0E94040B44D692E0692E92
:100A6C00892E90E0792E992EF8940000E2E0E09324
:100A7C00E900E091E800EB7FE093E8000000E091F2
:100A8C00E800EF77E093E8001E78F098077E91E09D
:100A9C009EBF9CEF9DBF789421CEF79B08950E943A
:100AAC00040B08959AE0D92EA8954CD5DD2019F4A5
:100ABC00F09BC3CF0895CEF79A35A1F31F79913AE5
:100ACC0081F01064923A69F09AE0D92EA895DD2055
:100ADC0039F038D5E6F79A3529F3953A09F0F7CF7E
:100AEC0027C008601061F09AAA27A0933B01A0933D
:100AFC003C01A0933E01BB27F7E0E0E096E0D92E45
:100B0C00DD20B1F01FD5E6F7F93008F4919311967A
:100B1C00BB23A1F3B23011F015FDF0CFA13071F76A
:100B2C0016FF04C015FD02C01062E8CF953A41F0E3
:100B3C008AE565D581EC63D585EA61D5077F089593
:100B4C00F7E0E0E0B5E0A0E091919D93B630E1F7DD
:100B5C008AE555D581EC53D585EA51D5077F0895A3
:100B6C003F925F936F930F930062F198F2989FE717
:100B7C0082EE0E94470B98D066F4332E832FF19AA5
:100B8C005ED5F19891D02EF4832FF19A58D5F19827
:100B9C0001C026C0532F9FE788EE0E94470B84D0DC
:100BAC006EF4832FF19A0E94250BF198432E7CD082
:100BBC002EF4832FF19A43D5F19801C011C0F1E0C6
:100BCC00E8E081D5532D7FD5532F7DD5542D7BD582
:100BDC005AE579D5B9D20F916F915F913F900895F5
:100BEC000C9423059FE78AEC4CD58AE308D582E068
:100BFC0020D30EF03BC00F7E3A3010F4832F04C08C
:100C0C0081E3FDD4832F8A50805D0E94050B532F06
:100C1C00552361F1513150F55F939FE788ED31D544
:100C2C009FE78AEC2ED58AE3EAD482E002D35F9167
:100C3C000EF01CC00F7E3A3010F4832F04C081E3F9
:100C4C00DED4832F8A50805D0E94050B0F7E3517F2
:100C5C0069F480E2D4D48FE6D2D48BE6D0D48DE084
:100C6C00CED4F1E0E4E05A952ED508950C942305EA
:100C7C0008609170F92F0E94A80AEEF7E92F9F2BBC
:100C8C0009F4F2E00E94BE0B0E94A80AEEF7077F5F
:100C9C00092E30912701409128010E94D60D3093E6
:100CAC00270140932801089582E0FCD226F44423C6
:100CBC0011F468940895E894089583E00E941F0944
:100CCC0016F40E94B90D089583E00E941F0926F4C2
:100CDC000E94B90D0E94D00D08950E94100956F47F
:100CEC000E94C10B03C00E94100926F430932A0104
:100CFC000E94D00D089583E00E941F090EF0089504
:100D0C00442371F580912701909128018F3F08F0C1
:100D1C0027C08F939F93E82FF92FFE5F00800092DE
:100D2C002A0101968093270190932801332389F09F
:100D3C003F938F939F930E94D00D9F918F913F91E2
:100D4C000196803031F080932701909328013A95D9
:100D5C0069F79F91909328019F9190932701089593
:100D6C006CCE0E9410090EF00895309331010E9450
:100D7C00130D08950E9410090EF0089530953695C4
:100D8C00309333010E94130D08950E9410090EF048
:100D9C000895309332010E94130D089583E00E9450
:100DAC001F090EF00895393C08F047CE30933001FE
:100DBC00343611F430E820C0393B10F096E015C001
:100DCC00363910F095E011C0383710F094E00DC0B2
:100DDC00353510F093E009C0323310F092E005C0C5
:100DEC003F3010F091E001C09927532F569556953E
:100DFC00350F390F08F43FEF30932F01089583E03E
:100E0C000E941F090EF00895442329F43A3518F472
:100E1C0030933A0110C011CE83E00E941F090EF0EE
:100E2C0008954423C1F73A35B0F73130A1F330932C
:100E3C003B01332309F031E030933E0133273093EB
:100E4C003C01089583E00E941F090EF00895309331
:100E5C003D0130933E0108953F934F93EF93FF93E1
:100E6C0080913D0180933E0180913C01992744275C
:100E7C0030913A01380F3A3508F033270E947F0C35
:100E8C00FF91EF914F913F9180913C01839590910F
:100E9C003B01891709F4882780933C01089583E06E
:100EAC000E941F090EF00895442309F021C0313827
:100EBC0008F030E883E70E94050B909126018091A1
:100ECC0025010E94A70986E70E94050BF5E0E09139
:100EDC002501EA9581910E949609E03031F03A950E
:100EEC0021F08CE20E94050BF5CF0E94040B0895B3
:100EFC00A4CD0F921F9283E40E94050B88E40E94FC
:100F0C00050B8DE30E94050B80912501682F9091B4
:100F1C0026010E94A70980E20E94050BF09128018E
:100F2C00E0912701FE5F508186E40E94050B89E663
:100F3C000E94050B8EE60E94050B8DE30E94050BAB
:100F4C00852F0E94960980E20E94050BF0912801E2
:100F5C00E09127016E2F51915F9384E50E94050B60
:100F6C0088E50E94050B8DE30E94050B852F0E94DE
:100F7C00960980E20E94050B82E50E94050B8DE329
:100F8C000E94050B5F91852F90912F01903841F0B5
:100F9C00899F812D803810F08FEF02C0000C881FC4
:100FAC000E94960980E20E94050B6F3F91F187E445
:100FBC000E94050B8DE30E94050B819190912F01EE
:100FCC00903841F0899F812D803810F08FEF02C04E
:100FDC00000C881F0E94960980E20E94050B6E3F50
:100FEC00C1F082E40E94050B8DE30E94050B808109
:100FFC0090912F01903841F0899F812D803810F00D
:10100C008FEF02C0000C881F0E94960980E20E949C
:10101C00050B0F938DE40E94050B86E40E94050BD3
:10102C008DE30E94050B0F7B809130010E94090A11
:10103C0085E20E94050B80E20E94050B83E40E946E
:10104C00050B83E50E94050B8DE30E94050B809137
:10105C003A010E94090A8FE20E94050B80913B0124
:10106C000E94090A8FE20E94050B80913D018F7747
:10107C000E94090A80E20E94050B84E50E94050B80
:10108C008DE30E94050B80912B010E94090A8EE2D0
:10109C000E94050B80912C010E94090A0F918DE092
:1010AC000E94050B1F900F900895992790932B0188
:1010BC0090932C0183E0BDD00EF0BFCC423008F0F1
:1010CC00BCCC5F9355279927442311F099E156E046
:1010DC00332361F03A3018F03A509395FBCF350F2B
:1010EC003A3010F03A5093955F9102C0352F5F91D2
:1010FC00903210F09FE139E090932B013A3008F0D8
:10110C0039E030932C0100244427990F892F990F33
:10111C00990F890F041E890F041E890F041E890F55
:10112C00041E890F041E890F041E880F001C330F28
:10113C00432F330F330F340F4427830F041E0092B9
:10114C002D0180932E0108959EE78CEE0E94470B93
:10115C009FE780E20E94470B9FE782EE0E94470BBD
:10116C00F1E0E8E00E945E0B902D0E945E0B802D5A
:10117C00892B11F0802D02C091E483E20F93006261
:10118C00F19A5DD2F198892F5AD29FE788EE0E948E
:10119C00470BF1E0EAE00E945E0B802D0E945E0B93
:1011AC00502D0E945E0B002011F0952F02C087E39A
:1011BC0090E0F79902C092E886E3582F892FF19AB4
:1011CC003ED2F198852F3BD280E219D218D29FE7FC
:1011DC008AEC0E94470B8DE312D2F1E0E4E00E940E
:1011EC005E0B00922301902D93959A3010F4892F69
:1011FC0004C081E304D2892F8A50805D0E94050BC4
:10120C008DE0FDD19FE78AE30E94470B0F91089573
:10121C000C94230506FF04C082E044D03EF403C0C6
:10122C0083E007D01EF4442311F4689408950C94C1
:10123C00230588D1F6F7332744278F9302C082D138
:10124C00F6F79D3039F19A3029F1903278F0B9F3F4
:10125C009C32A9F39E3299F39033E0F09734D0F49A
:10126C00913420F49A33B0F452D016F00C94230538
:10127C00330F441F532F642F330F441F330F441F5E
:10128C00350F461F6627390F461F8A95C1F668949D
:10129C008F91089500619F91891711F4E894089536
:1012AC00689408958F93332744274CD1F6F79D30DB
:1012BC0089F3973F11F49DE0EDCF9032E8F0A9F35C
:1012CC00903340F3973430F7913410F49A3310F78D
:1012DC0018D016F00C942305330F441F330F441F02
:1012EC00330F441F330F441F6627390F461F8A954F
:1012FC00E1F668948F9108950C942305913470F065
:10130C0002C0913420F0973448F4975305C09033C1
:10131C0028F090539A3010F468940895E894089546
:10132C009F93992706FF0AC08F9384E2F79967D1A0
:10133C000000F79BDED98F9166D001C064D09F91DD
:10134C0008950F930F7D5F936F933F92582F9923BE
:10135C0069F19732B0F011F4503198F087E2382EE1
:10136C0060E18827931540F011F4561728F0839507
:10137C000062561B9309F6CF8063F79940D1F79B17
:10138C00B8D983E0382E68EE8827931540F011F415
:10139C00561728F083950062561B9309F6CF80638D
:1013AC0005FF04C0F7992BD1F79BA3D988273324C9
:1013BC0064E6992311F4561728F083950062561BA6
:1013CC009309F7CF806305FF04C0F79918D1F79BF9
:1013DC0090D988276AE0561720F083950062561B37
:1013EC00FACF806305FF04C0F79909D1F79B81D927
:1013FC00852F8063F79903D1F79B7BD93F906F9131
:10140C005F910F9108950F9306FF1BC09F93982F28
:10141C0082958F7005FD41F0805D8A3308F0895FFD
:10142C00F799EDD0F79B65D9892F8F70805D8A3342
:10143C0008F0895FF799E3D0F79B5BD99F910F91E7
:10144C0008959F935F93982F8827943660F054E605
:10145C0080E38395951B9436E0F79F93F799CFD053
:10146C00F79B47D99F91882311F49A3068F05AE082
:10147C0080E39A3018F08395951BFBCF9F93F799D7
:10148C00BED0F79B36D99F91892F805DF799B7D045
:10149C00F79B2FD95F919F910F910895A89501FF0C
:1014AC004DC00D7F992790933701F09918C012FD0C
:1014BC000E94200E02FF13C00B7F90913B019923D9
:1014CC0071F080913D01882351F080913E01882379
:1014DC0031F08A9580933E0111F40E94320700FF8F
:1014EC0023C00E7F14FD06C00000F09B03C0F098D3
:1014FC002E9A5D9AD1D080911B018917A9F02E9854
:10150C005D9899279093D800A8950000FECFF89489
:10151C000E94780B81E08EBF8CEF8DBF7894A895DC
:10152C000E94800B0C94570380911501882331F095
:10153C008A958093150111F42E9A5D9A13FD0E94E1
:10154C00610E08958F93EF93FF93A8DF04FF04C0FF
:10155C00909138010F7E3CC0E894F82DE92D972D21
:10156C009E1721F4962D9F1709F444C09191F530E4
:10157C0011F4F2E0E0E08F2E9E2E5F936F93572DC7
:10158C00662D681430F009F005C0791410F0E1F004
:10159C0001C06D5F59196809623010F0503BA0F41E
:1015AC0010FF12C01E7FF8940000F2E0F093E900E7
:1015BC00F091E800FB7FF093E8000000F091E80068
:1015CC00FF77F093E80078946F915F9190933801D6
:1015DC00F79B07C003FD05C09B3718F4913608F044
:1015EC0090520F7E6894F09905C0E9E1E0931501E3
:1015FC002E985D98FF91EF918F9108958DE08F93C8
:10160C00F894000081E08093E900A8958091E800AF
:10161C0080FFFBCF8E7B8093E8008F918F9380931C
:10162C00F1008091E8008E7F8093E80000008091AB
:10163C00E8008F778093E80078948F9108958F93CA
:10164C0005FD02C080E2DBDF8F918F9382958F7056
:10165C00805D8A3308F0895FF19908C0F29B02C063
:10166C00803329F0803311F4F19B80E2C8DF8F9135
:10167C008F938F70805D8A3308F0895FC0DF8F9104
:10168C000895FF93EF93FC018591882311F0B7DF48
:10169C00FBCFEF91FF9108954F9B05C09927F79AC7
:1016AC00F498F39804C09FEFF798F49AF398089580
:1016BC0003D0009431960895F2BDE1BD002403944B
:1016CC000FBA00B40895509502D031960895A8959C
:1016DC00F894F2BDE1BD50BDFA9AF99AF999FECF92
:1016EC00789408959F939AEFA8950AD09A95E1F76C
:1016FC009F910895F7DFF6DFF5DFF4DFF3DF089550
:10170C009F9398EC992349F09F939F919F939F915E
:10171C000000000000009A95F5CF9F9108950024D9
:10172C0091E09093D70090EB9093D80000009F7DB0
:10173C009093D800000090629093D80090E199BDEE
:10174C00926099BD99B590FFFDCF9091D8009F7D87
:10175C009093D80099279093E00098E09093E20042
:10176C0092E0692E892E90E0792E992E7894089526
:10177C00FB5F31970895E0912501F0912601FF233D
:10178C0061F43196E0932501F09326010E94BE0B83
:10179C00F0932801E093270108950C942305F09110
:1017AC002801E09127015081FE5F0080902D9F3F22
:1017BC0049F00394008200922A01F250951719F413
:1017CC00008201C0F2500895F0912801E0912701A8
:1017DC005081FE5F0080902D9923A1F30A94EACFEB
:1017EC0082E00E941F09C6F53A3510F00C942305CF
:1017FC0013FFFECFAF93BF93EF93FF933F93F4E2AE
:10180C00F30FEE27A0E0B7E09BE5909337010E9421
:10181C00023FE0E89BE5909337010E94023F992735
:10182C00909337013F91332399F4F1E0E0E050912C
:10183C002D010E94690B50912E010E94690B5FEFE4
:10184C0006FD55270E946D0B3196522F0E94690B95
:10185C00FF91EF91BF91AF91089582E00E941F0913
:10186C00DEF73A3510F00C9423053323B1F4F1E094
:10187C00E0E00E945E0B00922E010E945E0B009233
:10188C002D010E94620B0F7B01FE006431960E94B9
:10189C005E0B902D907F2F70292BAF93BF93EF93FE
:1018AC00FF93F4E2F30FEE27A0E0B7E0A8950590C4
:1018BC0000940D92A030D9F7F5E0E0E0B7E0A0E09D
:1018CC00A8950C905081501559F080912E01909153
:1018DC002D01992321F4882311F4008201C07AD1BF
:1018EC0031961196F63061F7FF91EF91BF91AF9160
:1018FC0008953A3510F00C942305AF93BF93EF93F2
:10190C00FF93F4E2F30FEE27A0E0B7E0A895059063
:10191C0000940D92A138D9F7F5E0E0E0B7E0A0E033
:10192C00A8950C905081501559F080912E019091F2
:10193C002D01992321F4882311F4008201C04AD18E
:10194C0031961196E13861F7FF91EF91BF91AF910C
:10195C0008959FE788ED95DE0E94A80AEEF79F7D1B
:10196C00943411F00C9423058DE049DEF894F5E0E5
:10197C00E0E0B7E0A0E0992791939D93F630E1F772
:10198C00789408959FE788ED7CDE0E94A80AEEF714
:10199C009C3711F00C942305F894F1E0E4E0552702
:1019AC0092DEA8DEA7DEA6DE8DE00E94050BF89481
:1019BC00F5E0E0E099279193FB30E9F70F7B1F7B73
:1019CC00992790932A0190932B0190932C0190933B
:1019DC002D0190932E019093260182E380933A017E
:1019EC0090933B019093390184E180933D01939551
:1019FC0090932501909333019FEF9093320190E8DF
:101A0C0090932F0194E69093300195E090932801E8
:101A1C0090E09093270178940895309131013B32F6
:101A2C0038F4330F5FEF531B330F632F882742C0FB
:101A3C00353580F43B52432F4695469546956BEAD7
:101A4C00330F630F330F339533955CEA531B541BE1
:101A5C00882730C0303840F43555330F6FEF631B97
:101A6C00330F832F552726C03A3A80F43058432F32
:101A7C004695469546958BEA330F830F330F339576
:101A8C0033956CEA631B641B552714C0353D40F439
:101A9C003A5A330F8FEF831B330F532F66270AC02D
:101AAC00355D5BEA330F530F330F339533958AEA69
:101ABC00831B66271F92909133019F779923C1F066
:101ACC009F3709F490E84FEF451B499F412D000CBF
:101ADC00441F540F4FEF461B499F412D000C441FD0
:101AEC00640F4FEF481B499F412D000C441F840F7E
:101AFC00909132019F3F69F09695599F512D000CA2
:101B0C00551F699F612D000C661F899F812D000C4C
:101B1C00881F1F9060933501809336013091250109
:101B2C004091260150932A010E94D00D009035015E
:101B3C0000922A010E94C10B0E94D00D0090360128
:101B4C0000922A010E94C10B0E94D00D30932501F6
:101B5C0040932601E32FF42F0E94BE0BF093280133
:101B6C00E09327010895442329F0423088F433236D
:101B7C0079F402C0332361F03093250140932601A0
:101B8C00E32FF42FF5DDF0932801E093270108955E
:101B9C000C942305F0912801E091270100902A0173
:101BAC0000922A01F0932801E093270150815015EF
:101BBC0009F40EC0FE5F0082F25080912E019091CC
:101BCC002D01992321F4882311F4008201C002D045
:101BDC0078940895501908F45195002480912E01A1
:101BEC0090912D010AD0FD5F9083F3958083882717
:101BFC00F3958083F550146008954F923324441864
:101C0C0061E1001C551F6A9551F4969587958319CF
:101C1C009409802D952F08F401964F900895331C4C
:101C2C00441C381A490A20F4380E491E8894E9CF0E
:101C3C000894E7CF5F936F933F92F5E0E0E01B7F52
:101C4C008081FE5F9081891711F4F2501DC0F395CD
:101C5C005081F3956081F3953080360E08F45395DE
:101C6C003082891740F4850F20F0981710F014601B
:101C7C0009C0892F07C0851B20F0891710F014604C
:101C8C0001C0892FF55080833196E03009F0D8CF10
:101C9C003F906F915F910895599A93E09093CC0087
:101CAC009091C8009D7F9093C80099279093C9008C
:101CBC009EE09093CA000E94860BF8949091C90004
:101CCC00977B9093C9005B98539A78940E94860BEB
:101CDC005B9A14D01FD0F89495E0F92EEE249091D5
:101CEC00C90098649093C90099279093CE00177FF0
:101CFC00789408959F9392E00C94880B9F9390E1B5
:101D0C000C94880B9F9390EB0C94880B9F9390E012
:101D1C000C94880B9F9394E00C94880B892F8F70F4
:101D2C008F3011F0883050F40E94A80AEEF70E9410
:101D3C00A80AEEF70E94A80AEEF70895892F907F63
:101D4C0099F70E94A80AEEF790932001FBDBF6F7B7
:101D5C0090932101F7DBF6F79093220190912001EB
:101D6C00907F903A61F0903D51F0909120019F70DE
:101D7C0080912301981B29F010F0923010F00C94F4
:101D8C0023059093240150912001507F992331F029
:101D9C00503BA9F3503C99F3503E89F3503829F449
:101DAC0088278093220150E909C0503959F426FF45
:101DBC0010C080912201882309F46FC0823048F44E
:101DCC0088270DC0503B09F40EC0503C09F464C088
:101DDC0008C080912201880F8E3F09F48FEF60D0EC
:101DEC005CC086D05AC090912101992311F40C94B7
:101DFC002305933010F489D050C0973011F09830EF
:101E0C0011F49AD04AC0903131F444273091220118
:101E1C000E942D0742C0923111F4D8D03EC09331AC
:101E2C0011F4D9D03AC0953211F490D036C0983212
:101E3C00A8F111F4B5D031C0903480F129F430916F
:101E4C002201330F0C94BB06913429F430912201FA
:101E5C00330F0C94C406923429F430912201330FC1
:101E6C000C94CF069035D0F0943520F49235B0F424
:101E7C0021D013C0983510F432D00FC0903611F425
:101E8C0095D00BC0903711F49AD007C0973731F426
:101E9C009091220190932101A3D008950C942305D5
:101EAC0040912401309121010ED080932A010E948F
:101EBC00D00D0895409121013091220140554230BE
:101ECC0010F00C942305932F942B19F441E0332735
:101EDC0004C03F77469508F430680C94B90D909186
:101EEC00210191FD0E94C10B882790FD806402C0E6
:101EFC008091210190912201990F803408F091601A
:101F0C0090932A010E94D00D089580912101309167
:101F1C002201823051F0813069F499273A3018F05F
:101F2C003A509395FBCF0C947E0833279091220165
:101F3C000C947E080C9423053091220190FF3C599F
:101F4C00393C10F40C94DC060C94230530912201DE
:101F5C00332309F430E880EF0E947F038DE70E9461
:101F6C007F0383E70E947F039091260180912501D6
:101F7C000E94A70986E70E947F03F5E0E091250106
:101F8C00EA9581910E949609E03031F03A9521F062
:101F9C008CE20E947F03F5CF87EF0E947F030895A8
:101FAC004427309122010E94880608953091220125
:101FBC003A3518F444270C94370C0C9423053091C3
:101FCC0022013A35D0F744270C94FA0B4427309170
:101FDC0022010C9417074427309122010C940A0714
:101FEC0090912401992309F03EC0909121019130E8
:101FFC0019F40E946C3F36C0983019F40E94EA0B19
:10200C0031C0993019F40E94D50B2CC0903121F4B9
:10201C0078940E94320726C0953229F40F930E94BF
:10202C003B100F911FC0983711F42F7B1BC09937B1
:10203C0011F4206417C09F37B1F40E94A80AEEF780
:10204C000E94A80AEEF7592F507F0E94A80AEEF7BB
:10205C00692F0E94A80AEEF7503C29F46F3719F447
:10206C000E94BC0C08950C9423050F921F920F93A1
:10207C0080EF0E947F038DE70E947F0383E40E9420
:10208C007F0388E40E947F038DE30E947F0380918D
:10209C0025019091260155D980E20E947F03F09191
:1020AC002801E0912701FE5F508186E40E947F03A6
:1020BC0089E60E947F038EE60E947F038DE30E94D7
:1020CC007F03852F0E94960980E20E947F03F09186
:1020DC002801E09127016E2F51915F9384E50E94B6
:1020EC007F0388E50E947F038DE30E947F03852F89
:1020FC0017D980E20E947F0382E50E947F038DE363
:10210C000E947F035F91852F90912F01903841F0B1
:10211C00899F812D803810F08FEF02C0000C881F32
:10212C00FFD880E20E947F036E3F91F187E40E940A
:10213C007F038DE30E947F03819190912F01903852
:10214C0041F0899F812D803810F08FEF02C0000C78
:10215C00881F0E94960980E20E947F036F3FC1F0A6
:10216C0082E40E947F038DE30E947F038081909123
:10217C002F01903841F0899F812D803810F08FEF1E
:10218C0002C0000C881F0E94960980E20E947F0307
:10219C008DE40E947F0386E40E947F038DE30E94FE
:1021AC007F030F7B809130012ED985E20E947F0343
:1021BC0080E20E947F0383E40E947F0383E50E94F8
:1021CC007F038DE30E947F0380913A011CD98FE23B
:1021DC000E947F0380913B0116D98FE20E947F03FE
:1021EC0080913D018F770E94090A80E20E947F0353
:1021FC0084E50E947F038DE30E947F0380912B0175
:10220C000E94090A8EE20E947F0380912C01805D5E
:10221C000E947F0387EF0E947F030F911F900F9006
:10222C00089512011001020000080E0100000001C7
:10223C00090243000201008031090400000102027E
:10224C0000000524001001052401030004240207EA
:10225C000524060001070583031000400904010052
:10226C00020A000000070581024000010705020276
:10227C004000010009024300020100803109040002
:10228C0000010202000005240010010524010300D6
:10229C0004240207052406000107058303100040EF
:1022AC0009040100020A00000007058102400040F9
:1022BC00070502024000000A120355006E002000C0
:1022CC004B006E006F0077006E001C03550053002E
:1022DC0042002D00530069006D0070006C00650019
:1022EC0044006D00780000C20100000008000000EE
:1022FC0012010002010000080E0100010001090298
:10230C006500020100803109040000000101000099
:10231C000924010001090001010904010002010363
:10232C0000000724010001410006240201010006FF
:10233C002402020200092403010301020100092402
:10234C0003020401010100090581024000000000A4
:10235C0005250101030905020240000000000525C6
:04236C00010101006A
:0223FE000000DD
:10780000FFFFFF00FFFFFFFFFFFFFFFFFFFFFFFF87
:06781000FFFFFF5060FFC6
:10790000FFFFFF4040FFFFFFFFFFFFFFFFFFFFFF05
:06791000FFFFFF00FFFF76
:107A0000FFFFFFFF00FFFFFFFFFFFFFFFFFFFFFF85
:067A1000FFFF4040FFFFF4
:107B0000FFFFFFFF5060FFFFFFFFFFFFFFFFFFFFD3
:067B1000FFFF00FFFFFF74
:107C0000FFFFFFFFFF00FFFFFFFFFFFFFFFFFFFF83
:067C1000FFFF60FF60FFB2
:107D0000FFFFFF60FF60FFFFFFFFFFFFFFFFFFFFC1
:067D1000FFFFFFFF00FF72
:107E00000C9404035F938F939F93EF93FF93F4324B
:107E100020F4FE3710F00C942305F999FECF9091D1
:107E200037019B3511F00C94230599279093370166
:107E3000F89493E00E94423F91E10E94423F80E427
:107E40000D901D900094109491E00E94423F329654
:107E50008A95B1F7FF91EF91EF93FF9395E00E9420
:107E6000423F91E10E94423F87B786FF04C091E103
:107E70000E94423FF9CF7894FF91EF919F918F91AB
:107E80005F91089557B750FDFDCF97BFE8950895CE
:107E90000F7B0895006408950E9410097EF4F0910C
:107EA0002801E0912701FE5F9081930F08F49FEF76
:107EB000092E90932A01F2500E94D60D08950E9437
:107EC0001009E6F7F0912801E0912701FE5F90810B
:107ED000931B70F79927ECCFE0E0F5E0A0E0B7E066
:107EE00091919D93F630E1F71B7F08950D73696DB5
:107EF000706C65205553422F444D5820496E74656F
:107F0000726661636520666F722041726475696E86
:107F10006F204D6963726F202876312E313429002D
:107F200020286329323031352D323120572E5363CA
:107F300068656D6D6572740D00004A756D706572CF
:107F4000204F46463A41534349495F636D64536548
:107F500074202B204D696E69444D582C32353663A0
:107F6000680D4A756D706572204F4E3A4D4944490F
:107F70005F636D645365742C32353663680D0000A1
:107F80004A756D706572204F46463A4153434949E0
:107F90005F636D64536574202B204D696E69444D99
:107FA000582C32353663680D4A756D706572204FF6
:107FB0004E3A6F6E6C79204D696E69444D5820625F
:107FC00075742035313263680D004D494449206392
:107FD0006828312D31362900205265706561742082
:0E7FE00000005649443D0000205049443D0039
:00000001FF
